:1000000009C022C021C020C01FC01EC01DC01CC00E
:100010001BC01AC011241FBECFE9CDBF10E0A0E65F
:10002000B0E0ECE9F3E003C0C89531960D92A0363C
:10003000B107D1F710E0A0E6B0E001C01D92A137F2
:10004000B107E1F777D0A9C1DBCFF92FE82F262F31
:10005000372F4423A1F0E19912C09081B32FA22F32
:100060008FD1802D981729F09DBBF894E29AE19AE0
:100070007894415021F031962F5F3F4FECCF089597
:10008000B89A86BF82E48FBD2FEF94E688B78823A5
:10009000E9F328BF442339F4B898892F8A95F1F7FA
:1000A000B09909C0B89A88B78823E9F328BF6623B6
:1000B00069F3615059F71FBCB89884E68A95F1F747
:1000C0000895369A3699FECF85B19927089540E173
:1000D00060E070E081E690E0B8DF82B7813E38F5FD
:1000E000552029F0EEDF7816C0F75520F1F4E9DF4E
:1000F000861598F7352D552051F022B78091600074
:10010000820F912D911D96958795482E03C082B739
:100110008093600012BEBB9A88E08A95F1F7BB9885
:10012000532E509481E090E00895352DE6CF80E085
:1001300090E00895479A93E098BB83E287B983E8FB
:1001400086B98CE384BB80E1E1E6F0E0A0E0B0E0BA
:10015000182E1ED1809162008F3F11F41092620020
:10016000809163008F3F19F488E78093630080914A
:1001700064008F3F19F482E38093640093BF40E1F1
:1001800060E070E081E690E060DFB09BF8CFFF2494
:100190000FEF10E096DF8695801708F4082F1817E8
:1001A00008F4182FFA94B1F7312F300F812F9927C7
:1001B000801B910946E0959587954A95E1F7282F90
:1001C000882309F421E0732E720E632E621A12BE88
:1001D00055247DDF7CDF7BDF7ADF79DFB099FDCFCF
:1001E0008091690090916A00A0916B00B0916C00C1
:1001F0000196A11DB11D8093690090936A00A093A0
:100200006B00B0936C0039985CDF082F399A10911D
:1002100063003090620080916100992787FD90957E
:10022000252D33278217930709F051DF812F992756
:10023000602F772701977CD06FEF70E08BD0162F5F
:100240001F5F38983EDF389A682F60957727842D96
:1002500099276ED06BE171E07DD07727062F361697
:1002600008F4362E34DF8823A1F1B0992CC0932DE9
:1002700082B78917E8F325DF552019F0681618F4BE
:100280002EC0871560F1C198BB9AC39A95E0B99AC0
:100290000000B99884E08A95F1F79150C1F7BB98B6
:1002A000C398C19A0EDF7816D8F18615C8F150921E
:1002B0006100302E1150C9F0C4CF41E064E68FE0F8
:1002C000DFDE82E032C041E06AEF8FE0D9DE81E01C
:1002D0002CC040E060E58AE0D3DE83E026C040E049
:1002E00060E588E2CDDE85E020C010916400EFDE9D
:1002F000B099E3CF1150D9F780916D0090916E00C5
:10030000A0916F00B09170000196A11DB11D809366
:100310006D0090936E00A0936F00B09370002FCF8C
:1003200040E060E084E1ACDE84E08093650027CFAC
:100330005527002480FF02C0060E571F660F771F47
:100340006115710521F096958795009799F7952F7E
:10035000802D0895AA1BBB1B51E107C0AA1FBB1F1C
:10036000A617B70710F0A61BB70B881F991F5A9541
:10037000A9F780959095682F792F8A2F9B2F089544
:10038000E199FECFBFBBAEBBE09A11960DB20895C6
:0C039000F7DF01921A94E1F70895FFCF07
:00000001FF
